:1000000012C02CC02BC02AC029C028C027C026C0BF
:1000100025C024C023C065C421C031C01FC01EC07C
:100020001DC01CC01BC011241FBECFE5D4E0DEBF25
:10003000CDBF10E0A0E6B0E0EEE9F9E002C0059027
:100040000D92A036B107D9F710E0A0E6B0E001C0EC
:100050001D92AB37B107E1F7BFD39FC4D1CFDF9378
:10006000CF93CDB7DEB7EAE2F0E088ED8083E9E236
:10007000F0E08CE080837894CF91DF9108951F9217
:100080000F920FB60F9211248F939F93AF93BF934C
:10009000EF93FF93DF93CF93CDB7DEB780917800D6
:1000A00090917900019690937900809378008091E7
:1000B0007A00815080937A0080917A00882341F001
:1000C000ECE2F0E0A0917800B09179008C9180830F
:1000D000CF91DF91FF91EF91BF91AF919F918F9160
:1000E0000F900FBE0F901F901895DF93CF93CDB751
:1000F000DEB766970FB6F894DEBF0FBECDBF9B8B01
:100100008A8B7D8B6C8B4E8B1D821C821B821A828C
:100110008C899D8999238CF58C899D8990958195F1
:100120009F4F9D8B8C8B8A81282F30E08A899B89F9
:10013000FC01E20FF31F8DE280838A818F5F8A8347
:100140001CC08B81E82FF0E08C899D892AE030E08B
:10015000B901FCD3282F205DCE010696E80FF91FC8
:1001600020838B818F5F8B838C899D892AE030E08F
:10017000B901ECD3CB019D8B8C8B8C899D898A3006
:100180009105FCF68B81282F30E08C89482F405D4B
:10019000CE010696FC01E20FF31F40838B818F5F37
:1001A0008B830DC08B81282F30E0CE010696FC0199
:1001B000E20FF31F80E380838B818F5F8B839B81B2
:1001C0008C81891778F79B818D81981758F38B81E3
:1001D000282F30E0CE010696FC01E20FF31F1082BB
:1001E0008B818F5F8B838B81815089831B823BC086
:1001F0008981282F30E08B81882F90E0281B390BD4
:100200008C81882F90E02817390769F48A81282F7C
:1002100030E08A899B89FC01E20FF31F8EE2808324
:100220008A818F5F8A838A81282F30E08A899B891F
:10023000DC01A20FB31F8981882F90E09C0121501F
:1002400030408B81882F90E0281B390BCE01069619
:10025000FC01E20FF31F80818C938A818F5F8A8378
:100260008B818F5F8B839B818981981708F28A81AC
:10027000282F30E08A899B89FC01E20FF31F10824E
:100280008A818F5F8A838A899B8966960FB6F894E4
:10029000DEBF0FBECDBFCF91DF910895DF93CF9327
:1002A00000D00F92CDB7DEB79A8389836B8380919C
:1002B0007A00882379F489819A81909379008093D8
:1002C00078008B8180937A00ACE2B0E0E981FA811A
:1002D00080818C9380917A008823E1F70F900F90B2
:1002E0000F90CF91DF910895DF93CF9300D0CDB7DA
:1002F000DEB79A83898380917A00882389F4898183
:100300009A81909379008093780089819A8115D39E
:1003100080937A00ACE2B0E0E981FA8180818C932D
:1003200080917A008823E1F70F900F90CF91DF91B1
:100330000895DF93CF93CDB7DEB727970FB6F89424
:10034000DEBF0FBECDBF9F838E832E813F81CE0146
:100350000196B90140E0C9DECE010196C5DF2796BE
:100360000FB6F894DEBF0FBECDBFCF91DF910895D9
:10037000DF93CF9300D000D0CDB7DEB78BE1898378
:100380008BE58A838BE38B8388E48C83CE01019693
:1003900064E084DF0F900F900F900F90CF91DF916A
:1003A0000895DF93CF9300D00F92CDB7DEB78BE1E6
:1003B00089838BE58A838AE48B83CE01019663E08F
:1003C0006DDF0F900F900F90CF91DF910895DF9325
:1003D000CF9300D000D000D0CDB7DEB79E838D8301
:1003E00022C08D819E8101979E838D8380ED92E056
:1003F000A0E0B0E089839A83AB83BC830CC0898181
:100400009A81AB81BC810197A109B10989839A8343
:10041000AB83BC83000089819A81AB81BC8100974A
:10042000A105B10561F78D819E810097D1F62696D1
:100430000FB6F894DEBF0FBECDBFCF91DF91089508
:10044000DF93CF9300D00F92CDB7DEB79A83898325
:100450006B8399818B8189278B838B81882F90E097
:1004600082959295907F9827807F9827982F8B81EF
:1004700089278B838B81882F90E0382F22278981D1
:100480009A81892F9927282B392B8B8182958F7000
:10049000882F90E0282739278B81882F90E0880FBC
:1004A000991F880F991F880F991F822793270F90F4
:1004B0000F900F90CF91DF910895DF93CF93CDB739
:1004C000DEB72F970FB6F894DEBF0FBECDBF8C8777
:1004D0006D874E872F871B8281E48C8381E48D8317
:1004E0008C858E838D858F838E8588878F85898780
:1004F0001B861A86CE0104969A8389831B8213C0B9
:100500004A855B858B81282F30E089819A81FC01A7
:10051000E20FF31F2081CA01622F92DF9B878A8737
:100520008B818F5F8B838B81863050F389819A8199
:1005300068E0B4DE2F960FB6F894DEBF0FBECDBFD5
:10054000CF91DF910895DF93CF93CDB7DEB7279793
:100550000FB6F894DEBF0FBECDBF8C836D831B82B8
:100560001A8283E0898323C082E061E04C812D817F
:10057000A4DF109260008AE090E09B838A8308C029
:100580008A819B8101979B838A8381E090E01FDFB2
:1005900080916000882321F48A819B81009781F7F4
:1005A0008A819B81009719F081E08E830EC089813A
:1005B0008F838F81882311F081E08F838F819981D0
:1005C00091509983882381F61E828E8127960FB6DB
:1005D000F894DEBF0FBECDBFCF91DF910895DF93BA
:1005E000CF9300D00F92CDB7DEB78B8383E690E038
:1005F0009A83898380917500882371F58B8181347A
:1006000009F08DC080917600813409F088C08FEFA9
:1006100080937700109262001092610082E08093D4
:1006200075008B81809363008091610090916200DE
:100630006B8106DF90936200809361008B818093D1
:10064000640080916100909162006B81F9DE90936B
:1006500062008093610063C0809177008F3F09F052
:100660005AC080917500873010F580917500882FF1
:1006700090E0FC01ED59FF4F8B8180834091610038
:100680005091620080917500882F90E0FC01ED5937
:10069000FF4F2081CA01622FD3DE909362008093C6
:1006A0006100809175008F5F8093750038C08091E4
:1006B0007500882F90E0FC01ED59FF4F8B818083FE
:1006C000409161005091620080917500882F90E008
:1006D000FC01ED59FF4F2081CA01622FB1DE9093DA
:1006E00062008093610080916100909162000097A8
:1006F00069F4E981FA818281863041F4E981FA81E5
:100700008381813019F481E080936000109275003C
:100710001092770004C010927500109277008B81C0
:10072000809376000F900F900F90CF91DF910895F6
:10073000DF93CF93CDB7DEB7A1E3B0E0E1E3F0E024
:10074000808184608C93A1E3B0E0E1E3F0E08081FC
:1007500088608C93A1E3B0E0E1E3F0E08081806108
:100760008C93CF91DF910895DF93CF93CDB7DEB710
:10077000A2E3B0E0E2E3F0E0808184608C93A2E346
:10078000B0E0E2E3F0E0808188608C93A2E3B0E027
:10079000E2E3F0E0808180618C93CF91DF91089556
:1007A000DF93CF93CDB7DEB7A2E3B0E0E2E3F0E0B2
:1007B00080818B7F8C93A2E3B0E0E2E3F0E0808164
:1007C000877F8C93A2E3B0E0E2E3F0E080818F7E4C
:1007D0008C93CF91DF910895DF93CF93CDB7DEB7A0
:1007E00061970FB6F894DEBF0FBECDBF198237DC1C
:1007F000A5E3B0E0E5E3F0E0808181608C93A5E3C0
:10080000B0E0E5E3F0E0808182608C9391DF1982B3
:100810000DC08981282F30E0CE010296FC01E20F45
:10082000F31F80E4808389818F5F89838981883089
:1008300080F3E3E3F0E08081882F90E08170907096
:10084000009719F48EE78A830DC0E3E3F0E080811E
:10085000882F90E082709070009719F482E88A8364
:1008600001C01A82198239C08981282F30E0CE0157
:100870000296FC01E20FF31F40818981282F30E0AE
:10088000CE010A96FC01E20FF31F8081481711F197
:100890008981482F50E08981282F30E0CE010296CF
:1008A000FC01E20FF31F2081CE010A96FC01E40F48
:1008B000F51F208359DF8981282F30E0CE01029671
:1008C000FC01E20FF31F90818981692F3CDE8130AA
:1008D00009F466DF89818F5F89838981883020F2FE
:1008E000A8CF1F920F920FB60F9211242F933F9310
:1008F0004F935F936F937F938F939F93AF93BF9328
:10090000EF93FF93DF93CF93CDB7DEB7ECE2F0E048
:10091000808165DECF91DF91FF91EF91BF91AF9123
:100920009F918F917F916F915F914F913F912F9107
:100930000F900FBE0F901F901895FC0101900020A2
:10094000E9F7809590958E0F9F1F089597FB092ECC
:1009500007260AD077FD04D00CD006D000201AF468
:10096000709561957F4F0895F6F7909581959F4F0B
:100970000895AA1BBB1B51E107C0AA1FBB1FA617E6
:10098000B70710F0A61BB70B881F991F5A95A9F738
:0E09900080959095BC01CD010895F894FFCF9D
:00000001FF
